:100000008A110A120528000009000730990083169A
:10001000051085100511851505128512831205102E
:100020008510051105128512E830A0000330A100EB
:10003000E42105167620E830A0000330A100E42179
:100040009420AC012C080A3C031C3A28AD012D0871
:100050003B3C031C3428BC30A0000230A100E4214A
:100060000130AD07031C27281F3083050130AC0782
:10007000031C22281F3083059420AC012C080A3C65
:10008000031C5628AD012D083B3C031C5028BC30F6
:10009000A0000230A100E4210130AD07031C432879
:1000A0001F3083050130AC07031C3E281F30830539
:1000B0007620AC012C080A3C031C7228AD012D08E7
:1000C0003B3C031C6C28BC30A0000230A100E421A2
:1000D0000130AD07031C5F281F3083050130AC07DA
:1000E000031C5A281F3083053C28752805149030BE
:1000F000A0000130A100E4218516AD012D080B3CC4
:10010000031C8B28E830A0000330A100E42101305B
:10011000AD07031C7E281F30830585126430A000C4
:10012000A101E4210510080005149030A000013061
:10013000A100E421BE208421BA2084211F21842132
:100140000F218421B0208421C5209321D021C830E3
:10015000A000A101E42105100800AA21BD2108008A
:10016000BD21AA21AA21AA210800BD21AA21BD21C1
:10017000AA210800BD21AA21AA210800AA2108005D
:10018000AA21AA21BD21AA210800BD21BD21AA21A1
:100190000800AA21AA21AA21AA210800AA21AA218D
:1001A0000800AA21BD21BD21BD210800BD21AA2131
:1001B000BD210800AA21BD21AA21AA210800BD2134
:1001C000BD210800BD21AA210800BD21BD21BD21FE
:1001D0000800AA21BD21BD21AA210800BD21BD2101
:1001E000AA21BD210800AA21BD21AA210800AA2117
:1001F000AA21AA210800BD210800AA21AA21BD2107
:100200000800AA21AA21AA21BD210800AA21BD21F6
:10021000BD210800BD21AA21AA21BD210800BD21C0
:10022000AA21BD21BD210800BD21BD21AA21AA21ED
:100230000800BD21BD21BD21BD21BD210800AA218D
:10024000BD21BD21BD21BD210800AA21AA21BD21BA
:10025000BD21BD210800AA21AA21AA21BD21BD21BD
:100260000800AA21AA21AA21AA21BD210800AA21A9
:10027000AA21AA21AA21AA210800BD21AA21AA21D6
:10028000AA21AA210800BD21BD21AA21AA21AA21B3
:100290000800BD21BD21BD21AA21AA210800BD2140
:1002A000BD21BD21BD21AA210800AA21BD21AA216D
:1002B000BD21AA21BD210800BD21BD21AA21AA215D
:1002C000BD21BD210800AA21AA21BD21BD21AA214D
:1002D000AA210800BD21AA21AA21BD21AA21080026
:1002E000BD21AA21AA21AA21BD210800BD21AA2140
:1002F000AA21AA21AA21BD21080005110516503006
:10030000A000A101E4210800051105165030A0004D
:10031000A101E4215030A000A101E4215030A0004F
:10032000A101E4210800051105165030A000A1012B
:10033000E4215030A000A101E4215030A000A1012F
:10034000E4215030A000A101E4215030A000A1011F
:10035000E421080005150512053084000230AA00CA
:100360009930A0000230A1003530A2000030A30077
:100370001F22051105167D210800051505120530FF
:1003800084000230AA009930A0000230A100D230CF
:10039000A2000030A3001F22051105167D210800D0
:1003A00005150512053084000230AA009930A0001E
:1003B0000230A100EE30A2000230A3001F2205117E
:1003C00005167D210800E329A0080319EF29F6216D
:1003D000A00300000000000000000000E429A108C4
:1003E00003190800F621A103A003E4290C30A5009D
:1003F000A50BF829000000001230A200A20B052A6C
:10040000072207220000000008000722FE290D3005
:10041000A400A40B092A000008001030A802000163
:10042000031C013EA902031C0800162A0A30A80278
:100430000001031C013EA902031C0800162A2A0819
:1004400080042008A8002108A9000D220130A20282
:10045000031CA3032A0980052008A8002108A9007D
:100460000D22A208031D1F2AA308031D1F2A08002E
:02400E00C431BB
:00000001FF
